:020000020000FC
:100000000BC055C109C008C007C03AC105C004C033
:1000100003C002C001C000C09FED9DBFDD9A4FE24A
:100020004ABB49E047BBCC27DC9A0C2E0DE5409338
:1000300074000FEF302E0FEF56D155D154D153D15C
:1000400052D151D150D14FD14ED14DD10A95A1F7B6
:10005000C0C1552718E0869508F4560F5795879527
:100060001A95D1F753950895409174004F3271F16C
:100070004032F0F04F3318F5403368F45FE180EF21
:10008000451719F053958051FBCF40E040937B001A
:1000900080937A0020C050E38FE0451719F0539504
:1000A0000F96FBCF40E040937A0080937B0013C013
:1000B00040E040937B004FEF40937A000CC040E05B
:1000C00040937A004FEF40937B0005C040E040939F
:1000D0007A0040937B000895222795D208953091AD
:1000E00065009FEF931BE0917500E0937600E0932D
:1000F0007800909375003E3F21F499279093780003
:1001000002C09093780060916D0070916C006093D4
:100110006F0070936E0060916B0070916A00609345
:100120006D0070936C00609169007091680060933D
:100130006B0070936A005527772740917500609196
:100140007600461B570B552321F0413C28F441EC27
:1001500003C04F3308F04FE34093690050936800A9
:1001600008950F931F9373940FE3071511F408E09C
:10017000702E10917100110F0FEF011B38F00695D2
:10018000069517E0010F071508F001C0772417E066
:10019000711610F0DD9A01C0DD980F911F9108953E
:1001A000409169005091680060916B0070916A0005
:1001B000460F571F60916D0070916C00460F571FDE
:1001C00060916F0070916E00460F571F609175002F
:1001D000662351F060917B006623E9F0709178000E
:1001E000753578F0552331F05527509371005093B1
:1001F000720045C0842F509372002BDF5093710022
:100200003EC0552389F38FEF841B5093720021DF8A
:100210005093710034C060917A00552319F08FEF2C
:10022000841B01C0842F5093720013DF5093710020
:1002300090917A009C3018F18091750086956091BC
:10024000700007DF4427609171007091720077237E
:1002500051F08FEF861B850F741F682F772359F09D
:100260006FEF681B08C0650F741F7F3F21F0772375
:1002700011F077276FEF609371007093720008950B
:100280000F930FB70F93032F132F222748E01695D4
:1002900008F4200F279517954A95D1F7321608F4E0
:1002A000232DB1D133950F910FBF0F9118950F9357
:1002B0000FB70F93B69901C006C0002702BF0F9178
:1002C0000FBF0F91189502B7009374000F910FBFE5
:1002D0000F911895B29B08951BE01A95F1F733958D
:1002E00000000000F7CF15E02EE52A95F1F71A95EA
:1002F000D9F70895C09A0BD0332339F01BE01A9533
:10030000F1F73A9500000000F7CFC09808951AE081
:100310002FEE2A95F1F71A95D9F708953327DEEFD6
:10032000262D2FBD282D2BBD24E029BFD31799F0F2
:100330004599FCCF30936500132E1394212C239400
:100340004599F4CF1316E1F7CC9B07C04599EECF42
:100350002316E1F702C03093650022272FBD2EBD82
:10036000089500E1C39A10E1DB9A1A95F1F70000B5
:10037000DB9820E22A95F1F700000000DB9A1FE1EC
:100380001A95F1F7000000000A9591F7DB98C398E1
:1003900008955CB351FDFDCF4EBB8DBBE29AE19A4F
:1003A00008955CB351FDFDCF4EBBE09A5CB350FDA8
:1003B000FDCF8DB308955A9559F458E0A7FF02C0B8
:1003C000DD9801C0DD9AAA1F6A9511F4AB2F66E093
:1003D000089582DE33270027772499DF04E8602E12
:1003E00001E3802E0027009371000093720004E067
:1003F00003BF00E40BBF01E005BFCC9955C0DD98F9
:10040000CC9BFECF58E066E0ACE7BCE7B29BFECFEA
:100410007EDF60DF30937D00932F6CDFCCDF3327EE
:10042000CC99F4CFDD98CC9BFECF58E066E0ACE5EC
:10043000BCE5B29BFECF6BDF4DDF30937E00932F88
:1004400059DFB9DF3327CC99F4CFDD98CC9BFECFB1
:1004500058E066E0A5E5B5E5B29BFECF58DF3ADF90
:10046000932F48DFA8DF3327CC99F6CFDD98CC9BBC
:10047000FECF80917D0070917E00781720F0981B50
:1004800038F4992705C0891B10F4992701C0982FCB
:1004900041E080917D007DDF42E080917E0079DF48
:1004A00043E0892F76DFDD9ADD9A4427409371007F
:1004B0004093780040937700409375004093760016
:1004C0004093680040936A0040936C0040936E0034
:1004D0004093690040936B0040936D0040936F0020
:1004E00040937900332743E05CDF8093700041E064
:1004F00058DF80937D0042E054DF80937E0045E02A
:1005000050DF40EE46E04DDF80936600382E80914C
:100510007E0070917D00871708F41DC07894B29B0F
:10052000FDCFF5DED7DE3093630080D030916400DC
:10053000932F7894DFDE15DFD6DED5DED4DED3DE72
:10054000D2DEECDECCDD2CDEC7DD3327032E3CD043
:100550008BDDC1D0E3CF7894B29BFDCFD8DEBADE7D
:10056000309363008DD030916400932F7894C2DE75
:10057000F8DEB9DEB8DEB7DEB6DEB5DECFDEAFDD83
:100580000FDEAADD3327032E1FD06EDDA4D0E3CF0C
:1005900005E003BF04E8CC9B04E8602E05E4802E50
:1005A000E0DEA1DEA0DE9FDE9EDE9DDEB7DE97DD13
:1005B000F7DD92DD3327032E07D0FBEA02B7F017F1
:1005C000E9F7002702BFE6CF0F931F93739400E271
:1005D000071510F404E0702E009165000E3F69F0DD
:1005E000002369F00695069517E0010F071508F03E
:1005F00001C0772417E0711610F0DD9A01C0DD9874
:100600000F911F910895D9981F9318E0D898DA9AFE
:10061000DA98DA9ADA9827FDD89ADA9AD898DA9896
:10062000220F1A95C1F7D99A1F910895CC9B25C026
:10063000D0917100E091720070917E00EE2329F05C
:100640003D1B28F470917D0015C03D0F98F0731785
:1006500088F070917D00731768F470916300D091F9
:100660007E00D71738F0D0917D007D1718F03093B9
:10067000640002C07093640008959FEF392EF7CF95
:10068000CC9B26C0D0917100E091720070917D00EA
:10069000EE2331F03D0FC8F005C070917E0015C00B
:1006A0003D1BD8F3731788F070917E00731768F4C0
:1006B00070916300D0917D00D71738F0D0917E0003
:1006C0007D1718F03093640002C0709364000895A1
:1006D0009FEF392EF7CFCC9B0AC090916600391658
:1006E00049F03092660046E0832D53DE03C09091BE
:0606F0006500392E08959B
:00000001FF
